:0A00060000308A002C28000045306D
:100010008400000803191B280130F800F701F70BD2
:100020000F28F80B0E284A30F700F70B15280000B0
:100030000000800B0C288A112A2805150511303084
:100040004302C400333044078400000886000530B2
:10005000C50007288A11662884011F30830583168E
:100060001F08C0399F009B01073083129F007E301C
:10007000B3000C30B400B630B5009E30B600CC30C2
:10008000B700DA30B800FA30B9000E30BA00FE30EE
:10009000BB00CE30BC003830BD003030BE00333045
:1000A000BF00C00183168501860183128501860188
:1000B00085148510C1014108023C031C68283D30AD
:1000C000410784000008C200C3001D28C10A5B2844
:0400D0005828630049
:040000008A01032846
:00000001FF
